:030000000219FDE5
:03000B000200AA46
:03002B0002015C73
:03005B000202F6A8
:030073000202E3A3
:1000800002030406080C10182030406080040608A3
:100090000C10182030406080A0C00003070F1F0D17
:1000A0000D04050D050305030302C2AFC0D0C0E077
:1000B000206214E5256009E473E525F4F58AD2622F
:1000C000D0E0D0D0D2AF3285268AC262E526F46075
:1000D0002F30682520720DD0E0D0D0C2B1C287C2C7
:1000E00081D2AF32C2B1C287C281206F0C206509B4
:1000F000740AD5E0FDE57B4280D0E0D0D0D2AF32AB
:10010000758A00C28DD26201F901B9306805206597
:1001100002D2B101B9306805206502D28701B93039
:100120006805206502D28101B9C28230680A206563
:10013000077408D5E0FDD2B101B9C28630680A2043
:1001400065077408D5E0FDD28701B9C28030680A1E
:100150002065077408D5E0FDD28101B9C2AFC2ADF8
:1001600053E6EFC0D0C0E0D2D3D2AFC2CEE52A6012
:100170000720744F152A21C37800790020742EE5DA
:1001800080307E01F430E50278FF53DACF207E0321
:1001900043DA20307E0343DA10C2D8C271E58030E2
:1001A0007E01F430E50279FFC3E89970CB3061033A
:1001B000752A18207403752A18885CD270E86003C9
:1001C000755F0020740DE52B6004152B21D343DAF5
:1001D00001C2D82070024142A85C206102C2702096
:1001E00074367982B70431C3E894F0400374F0F8B0
:1001F000E8C4540F28F87984B703024118C313C325
:10020000138721200802C313200A06C3C898F841A7
:100210001828F8500374FFF88822E52D5406602250
:10022000206B1FE536C333C333F8E564C313C31330
:10023000F9C3952240028922E82522F52250037550
:1002400022FF7882B60459852224A824C3E5249588
:10025000614002A861C3E895634002A8638825E570
:100260006670024193C3E8AA669A5003E8FAE4F97B
:10027000EAC333FBE568F45B29400D2567F8E567C1
:1002800060021567400B41930AC3E5679A50020567
:100290006778FF8826C26FC3E52694F84002D26FC4
:1002A00020CF0AD0E0D0D043E610D2AD32C2CF0585
:1002B0003A7801E52A6005307402152AC3E55C949A
:1002C000014005755F0041D9756000756900E55F03
:1002D0002401F55F5003755FFFD0E0D0D043E610F6
:1002E000D2AD32C2AF53E67F7592FA7593FFC2600A
:1002F000759104D2AF32C2AF53E6EFC2ADC0D0C0E9
:10030000E0C0F0D2D3D2AFA8FBA9FCC2D8307102B2
:10031000615D53DACF207E0343DA10307E0343DA87
:1003200020D271E580307E01F420E5026134882717
:100330008928A18A53DACF207E0343DA20307E0356
:1003400043DA10C2D8C271307402A1767800E58019
:10035000307E01F430E502A176885CA15E53DACFED
:10036000207E0343DA20307E0343DA10C27120611D
:1003700002813653DACF207E0343DA10307E034306
:10038000DA20C2D8D27188578958C3E89555F8E960
:100390009556F97B007E087A00C3E8948CE99400B6
:1003A0005005755B008128882178A2E6A821605558
:1003B000C3E894C8E994005008E4D2E4FB7A0A81C7
:1003C00003C3E89468E994015008E4D2E3FB7A0F90
:1003D0008103C3E894D0E994025008E4D2E2FB7AA6
:1003E0001E8103C3E894A0E994055008E4D2E1FB20
:1003F0007A3C8103C3E89498E994085008E4D2E079
:10040000FB7A787E00C3E89559FCE9955AFD30E700
:100410000AECF42401FCEDF43400FD755B00C3EC40
:100420009AED9E5003755B018859895A8557558509
:1004300058567802A15EC3E89527F8E99528F93067
:100440007C02A142307B02A142307A02A13B20759E
:10045000028159E9FDE8FC8178E9C313F9E813F852
:10046000307902A13BE9C313F9E813F8307802A10F
:0F0470003BE9C313FDE813FC20612CC3EC941C83
:10047F00ED94024002818FED701EC3EC94C85018AA
:10048F000529E52970021529C3E529940A5002A10F
:10049F0076755C00D270A176E529600215297888FF
:1004AF00E6F97400207F087896B90302789EE62457
:1004BF00FAFEE43400FFC3EC9EFCED9FFD9208B9F9
:1004CF000310A2085007207609D27681E130760218
:1004DF00C276A2085016B9030DECF42401FCEDF41A
:1004EF003400FD0204FB78007900A142B90315EC3A
:1004FF0033FCED33FDC3EC940AFCED9400FD500486
:10050F007C007D00C3EC94FFED9400400678FF79EA
:10051F0000A142EC8572F0A4C5F0A2F733F8790080
:10052F00400302055E78FF790002055EE9C313F907
:10053F00E813F8307C0EE9600278FFC3E81338F84F
:10054F00E43400F9C3E894FFE99400400278FF888F
:10055F005CD270206102A176741FF4552F4BF52FDA
:10056F00C274EB7002D274752A18307403752A0A9C
:10057F00306102A18A20740353DAFE207403752BB5
:10058F0006D0F0D0E0D0D0D2AD43E61032790102E0
:10059F0005BA79030205BA790A0205BA791E02056E
:1005AF00BA79640205BA79C80205BA7817E4D5E0BA
:1005BF00FDD8FAD9F6227A147B780205E17A107BFE
:1005CF008C0205E17A0D7BB40205E17A0B7BC80240
:1005DF0005E1E573D5E001227902E4C286D5E0FD9D
:1005EF00D287D5E0FDC287D5E0FDD286D5E0FDE903
:1005FF0020E002D2B130E002D281E573D5E0FDE90F
:10060F0020E002C2B130E002C2817496D5E0FDD97C
:10061F00C9EAF8D5E0FDD8FBDBB8C28622C37C005F
:10062F007D0075F00005F0EA33FAEB33FB50F6EB83
:10063F0013FBEA13FAC3E9FFE8FEE89AF8E99BF91E
:10064F005004EFF9EEF8B3EC33FCED33FDD5F0DFEA
:10065F00EDF9ECF822E889F08A20D2D4F8A9F07BE2
:10066F000030F70B7BFFF42401F8E9F43400F9E8CC
:10067F008520F0A4ADF0F8E98520F0A4AFF0FEEDF1
:10068F002EF974003FFA7C04C3EA13FAE913F9E870
:10069F0013F8DCF48BF030F70AE8F42401F8E9F4EE
:1006AF003400F9E889F0C2D4F8A9F0227882B604B0
:1006BF0003020716C3E55C940140030206E085229E
:1006CF0024E4F544F545F546F547F548C26E0207B3
:1006DF00167882E6FCD26EE522F523783879C7AA20
:1006EF0040AB41C3EB13FBEA13FAEC146013C3EBFB
:1006FF0013FBEA13FAEC14146007C3EB13FBEA13B2
:10070F00FAD12C8844894522C3E5449523F8E54561
:10071F009400F9500CC3E89480E994FF4016020747
:10072F0047C3E8947FE994005003020747787F7925
:10073F0000020747788079FF8849894A22E54925D1
:10074F0046F8E54A3547F9854A20E4300701F43584
:10075F0048FA30E709C3EA94F04015020785C3EA67
:10076F00940F500302078578FF79FF7A0F020785F0
:10077F00780079007AF0C3E5249561500AC37401BB
:10078F009524500B0207A3E54A20E70E0207A3E5C5
:10079F004A30E706884689478A482278A5E6FAC391
:1007AF00E54933F8E54A33F9D164E930E70BC3E89B
:1007BF009480E994FF4013E1DDC3E8947FE994004E
:1007CF005002E1DD787F7900E1DD788079FFE82064
:1007DF00E715C3E52398F84009C3E89401400302E5
:1007EF0008047801020804E8F424012523F84003E3
:1007FF0002080478FF884B2278A6E6FAA847A94892
:10080F00120664E930E70CC3E89401E994FF40163F
:10081F00020839C3E894FFE99400500302083978BD
:10082F00FF7900020839780179FFE920E715C3E560
:10083F004B98F84009C3E89401400302086078011F
:10084F00020860E8F42401254BF8400302086078A1
:10085F00FF88242278FF20692879A1E76023E541EA
:0E086F00601F74FF8541F0848539F0306A0304
:10087D0075F005A4F8C5F0600278FFC3E8956450E3
:10088D0002A864886322C3E5409440E5419401E5E4
:10089D006350031401A4046002F563220208AC2224
:1008AD0075E890227883E6FF30EDF9A8BDA9BE0565
:1008BD0070C3E57094084052757000E9FA79A0E7AD
:1008CD006044EA7007E571601B0208E5C3E89571A5
:1008DD006010E5715006600C140208F10460F90215
:1008ED0008F1E571F571C394A8401B7561C0C394FF
:1008FD00054013756180C39405400B756140C39429
:10090D0005400375610075BB0622E5612410500298
:10091D0074FFF5617982B70402213EC3A861E52415
:10092D00985002A824C3E895634002A863882588DF
:10093D0026E570B4070375BB1E22743279A787F0C4
:10094D00A4C5F0A2F733F8C3E895614002A8618809
:10095D00228824882588268864227540007541F0F8
:10096D0022C2AF75C820A8CCA9CDAA3A30CF010AB2
:10097D0075C824D2AFAB3BAC3C883B893CC3E89BEC
:10098D00F8E99C206908F9306602417F21D9AD3D17
:10099D008A3DF9EA9DFA600678FF79FF21BEAE3EE9
:1009AD00AF3F8B3E8C3FA83BA93CC3E89EF8E99F27
:1009BD00F9C3E54113FBE54013FAE82AF540E93B9D
:1009CD00F54150067540FF7541FF4126AA40AB41E8
:1009DD00AC40AD417E047F02C3EB9404400D1E1F5D
:1009ED00C3EB94084005206A021E1FC3ED13FDECF6
:1009FD0013FCDEF7C3EA9CFAEB9DFBEF6009C3E93C
:100A0D0013F9E813F8DFF7EA28FAEB39FB8A408B84
:100A1D004150067BFF8B408B41C3EB94025002D2B9
:100A2D00663069047F0341517892E6FFC3E5379440
:100A3D008240110FC3E53794A040010FC3EF940618
:100A4D0040027F057E02E541C4540FF9E541C454CF
:100A5D00F0F8E540C4540F28F8C3E89EFAE9940075
:100A6D00FB4009C3EA9402EB940050047A02E4FBC4
:100A7D0041CBAA40AB41EBC4FEEAC4540F4EFCC3BC
:100A8D00EA9CFAEB9400FBC3E813C313F8EA28FAC7
:100A9D00EB3400FB8A408B41C3EB94024002C266EB
:100AAD007802EBC4FE7B00EAC4540F4EFAC3EA98F9
:100ABD00FA4005C3940250027A027892E6FF306044
:100ACD000241CB855192855293D26043E680C3E4B7
:100ADD009AF8E49BF93066026157E8FAE9FBD3E92D
:100AED0013FDE813FC88518952C3EF94036038EF6E
:100AFD0020E00DE82CF8E93DF9ECFAEDFB020B20B6
:100B0D00E828F8E939F9C3E82402F8E93400F97A5C
:100B1D00FE7BFFC3EF9403400E8A538B54884D899F
:100B2D004E8C4F8D50618B885389548A4D8B4E8CD2
:100B3D004F8D503069127553F07554FF754FF07528
:100B4D0050FF7551F07552FF618BE8FAD3E813FC35
:100B5D008851C3EF94036020EF20E007E82CF8ECF8
:100B6D00FA6177E8282402F87AFEC3EF940340086F
:100B7D008A53884D8C4F618B88538A4D8C4FE56815
:100B8D00C3335002646BF5683060026195753402B1
:100B9D00D26043E680E52D54066034A840A941C3D8
:100BAD00E913F9E813F8C3E913F9E813F830690408
:100BBD00E92440F9C2AF53E67F759100C3E498F57F
:100BCD0094E499F595759104D26043E680D2AF22F5
:100BDD00D264754300752000306C03752040020B04
:100BED00FCD264754300752040306C03752000788D
:100BFD00017901206620E52D54066002C264791446
:100C0D00E541C313700104F8C39414400278143005
:100C1D006904781B791B206010E543600C30690373
:100C2D00D53404D26D81A6719D0543E59B5440B525
:100C3D002002819030690908C3E899400118812389
:100C4D0020640A08C3E899400261FC8123C264C292
:100C5D00AF53E67F7591003066127594007595F867
:0E0C6D00759104D26043E680D2AF61FCE54190
:100C7B007EFFC3334005C3334001FEC3E49E75942E
:100C8B0000F595816DC3E5339401500261FC30642E
:100C9B000261FCD80281A48123C26DC2AF53E67FEF
:100CAB00759100855394855495759104854D928566
:100CBB004E93D26043E680D2AFE52D5406600820F8
:100CCB006A020533020CE2306D0D206C0A206407BA
:100CDB00158115810215B52278003064027801E583
:100CEB003775F007A4F9E5F028F5F0E9A2F013A2A7
:100CFB00F113A2F213F537C394785003753778C309
:100D0B00E53795384008D265C2B1C287C2813060E1
:100D1B0002A119854F92855093D26043E680222021
:100D2B007D16C2AF754202C286D282306202D28178
:100D3B00D2AF759F02020F1AC2AF754202C286D2A2
:100D4B0080306202D2B1D2AF759F02020F1A30729D
:100D5B0043207D20C2AF75420390013A757B40C2A0
:100D6B0081C280306204D287A177D286D2AF759FC1
:100D7B0003020F1AC2AF75420390013A757B40C252
:100D8B00B1C282306204D287A197D286D2AF759F4F
:100D9B0001020F1A207D17C2AF754203900115C2D5
:100DAB0081306202D287D2AF759F03020F1AC2AF96
:100DBB00754203900115C2B1306202D287D2AF7572
:100DCB009F01020F1A207D16C2AF754204C282D258
:100DDB0080306202D287D2AF759F01020F1AC2AF69
:100DEB00754204C280D282306202D287D2AF759F25
:100DFB0003020F1A307243207D20C2AF754205905B
:100E0B000129757B04C287C286306204D2B1C11D31
:100E1B00D282D2AF759F02020F1AC2AF75420590F4
:100E2B00014B757B01C287C286306204D281C13D02
:100E3B00D280D2AF759F02020F1A207D17C2AF75F9
:100E4B00420590010BC287306202D2B1D2AF759FBF
:100E5B0002020F1AC2AF75420590011FC2873062A2
:100E6B00EBD281D2AF759F02020F1A207D16C2AF53
:100E7B00754206C280D286306202D2B1D2AF759F64
:100E8B0003020F1AC2AF754206C282D286306202CB
:100E9B00D281D2AF759F01020F1A307244207D2090
:100EAB00C2AF75420190014B757B01C2B1C282305A
:100EBB006204D281C1C3D280D2AF759F01020F1AD7
:100ECB00C2AF754201900129757B04C281C280308B
:100EDB006205D2B1020EE4D282D2AF759F03020F2C
:100EEB001A207D17C2AF75420190011FC2B130624B
:100EFB0002D281D2AF759F01020F1AC2AF754201A8
:100F0B0090010BC281306202D2B1D2AF759F03C286
:100F1B006522900109757B00C2B1C287C281C28272
:100F2B00C286C280C262227880760908760908766A
:100F3B00040876FF0876030876FF0876090876031F
:100F4B00087601087601788C76010876FF0876FF23
:100F5B000876FF0876FF0876FF0876030876FF0809
:100F6B0076FF0876FF0876250876D008762808766F
:100F7B00500876040876FF08760208760008767A21
:100F8B000876FF08760108760108760008760308D4
:100F9B007600227887E6FFC272BF0302D27278888E
:100FAB00E6C394036008C27DE630E102D27DC27EC7
:100FBB007889E630E102D27EC3EF94026008758E29
:100FCB0001D273020FD6758E00C273227880E6149D
:100FDB009000809378A5F67881E614900080937842
:100FEB00A6F67886E61490008D9378A7F67886E6B9
:100FFB00F539C394025003753902789CE67538FFB6
:10100B00B402037538A0B4030375388278A3E614D1
:10101B0090009A93F566120F1D22C2B3789DE6607D
:10102B0002D2B3227896E6FA7897E6FB7888E6B494
:10103B000305C3EB940EFB307F047A007BFFC3EBFD
:10104B009AFCC3948250027C827572000572EC8507
:10105B0072F0A4C3E5F0947D40F222D27F112F12DF
:0E106B0005AB1205AB7A007B007C101205A1CC
:10107900E55C2AFA74003BFBDCF37C04C3EB13FB4D
:10108900EA13FADCF7FEC27F112F22757C00757D09
:1010990000E5EF20E6037520000520903DFFE520DF
:1010A900146006901FFF1460009304600375EF1627
:1010B90053D9BF7581C043FF8012059C75EF064364
:1010C900B203E5B3240220E70DF521E5B120E006DE
:1010D9008521B343B101120F1D75803875A4C775F9
:1010E900F1FF75D4DF7590FF75A50075F20075D510
:1010F9000075A0FF75A60075F30075D60075B0E4FC
:1011090075A71B75F4FF75E241120F1DE4F8F6D8B7
:10111900FD756801120F32121606789886737530BC
:1011290001C2AF1205B51205C51205AB1205CC12E5
:1011390005AB1205D31205ABC2AF757C00757D00F6
:1011490078FA79FA308507D9FBD8F7021C00120F13
:101159009E120FD71125112F78988673120F1D75BE
:10116900881075890275C82475910475D84075A8C9
:101179002275B80275E690759B80759D0075D10E34
:1011890075BC5875BB0675BA1F75E88012059CD2E7
:10119900AF1208A975360053DACF207E0343DA204F
:1011A900307E0343DA1043DA01C2D8C2711205B5A1
:1011B900D2617B037A0CE55B70077A0CDB030211C1
:1011C900411205AB207003021141C270E55CC39462
:1011D9000240E1E52F541F855E5DF55EB55DD5DA08
:1011E900D5C26153DACF207E0343DA20307E034330
:1011F900DA10C2D8C27178A2E67008D274E52F5409
:10120900E0F52FC2757529001205B0307409C3E5E0
:1012190029940A4002D2751205A178023074027825
:1012290000C3E55C9840F0C2AF1205C51205C512AE
:1012390005C5D2AF1205B5754C007888E6B403022E
:1012490061361205A1788CE6C39401500302133666
:10125900E530C394015003021336757CA5757DF101
:10126900207435C3E55C94FF5003021336C2AF12F4
:1012790005DAD2AF1205B0C3E55C940150EFC2AFF5
:101289001205C51205A61205C5D2AF1205B0C3E5F0
:101299005C94FF40E90217BE7F02D27F112F12052D
:1012A900B0C2AFC27F112FAE5CC3E55C947FD2AFF1
:1012B9005002614612059CC2AF1205DAD2AFDFDADD
:1012C9001166C3EE7897F61205B51217417F0AD257
:1012D9007F112F1205B0C2AFC27F112FAE5CC3E5DB
:1012E9005C947FD2AF50E612059CC2AF1205C512BD
:1012F90005A61205C5D2AFDFD61166EE240378968E
:10130900F6F87997E7C394824003985006E8248257
:101319007897F61205B51216541217701205B01106
:101329002FC3E55C94FF500241630217BE757C0030
:10133900757D00C3E55C954C4003855C4C1205B096
:1013490078017988E7B403027805C3E55C9840021F
:101359004143C2AF1205DA1205DA1205DAD2AF1229
:1013690005B5753000E4F531F5320531E531F47034
:101379003F0532789AE67819146012783214600DB4
:10138900787D14600878FA146003753200C3E53279
:1013990098401D120F1D12059C1532753100789960
:1013A9008673C2AF1205DAD2AF789886731205B088
:1013B9001205A6E52A7005307402214178012074CE
:1013C900027806C3E55C9840A17888E6C394036077
:1013D900031205B0E52A7003021141C2AF120F1DB5
:1013E900E4F522F523F524F525F526F567D2AF783E
:1013F90085E6C333F565E4F544F545F546F547F566
:1014090048F570F52CF52DF53775700875BB1E126A
:10141900059C1208AD30EDFDA8BDA9BEE97001F823
:1014290088711208B175700875BB1E120F9EC2AF84
:101439007561FF120947852261852262852263D27F
:10144900AF7522017524017525017526018560692D
:10145900756A017888E6B40307C27D307602D27DC9
:0D146900D268D269753300120E76120EA5FE
:1014760012096712096E12096712096E12096712BC
:101486000BEE1206BB120CE3120D2A12096E120B9A
:10149600DD306E03120717206603120863306603F9
:1014A600120893120CE3120D5912096E120BEE304C
:1014B6006E0312074C120CE3120DD012096E120BBA
:1014C600DD306E031207AA120CE3120DFF12096E2D
:1014D600120BEE306E03120807120CE3120E761290
:1014E600096E1208AD120BDD120CE3120EA51208DE
:1014F600B112096E306932856461856462856069FE
:10150600756A0179187A0CC3E53399400FC269D21E
:101516006A8A3585646185646302152FC3E55C9428
:101526000140030214850215BD306A25206C22E5B0
:1015360035147006C26AD26B8185F535C3E55C94B5
:101546000140030214857888E6C3940360030215FC
:10155600BD75360078FA79A4E760027803C3E55FC3
:10156600985054307404E52A604D7888E6B4031721
:10157600207D05207607A18D307602A18D206C078F
:10158600D26C85646181C478F0306C0585646178BD
:1015960020C3E5419850028185306C1BC26CC27D28
:1015A600307602D27DD26A753512856461818505F1
:1015B60036E55C6002A1C0753600C2AF120F1D7819
:1015C60087E6FE7602120F9E7887EEF6E4F522F5A0
:1015D60023F524F525F526F565752C00752D00D225
:1015E600AF1205B0120F1D78A4E66006D2B1D287FD
:1015F600D281307409C3E536940440022141616EFC
:10160600901A0D7820121696E520B4550CA31216E2
:1016160096E520B4AA03021634757CA5757DF112F1
:101626000F32121654757C00757D00021653901AFF
:101636000378807B0A121696A308DBF9901A0F78B6
:101646008C7B19121696A308DBF9901A2822C2AFD2
:101656001216D91216B6901A00740E12169BA3749F
:101666000912169BA3741512169B901A0378807B99
:101676000A12169AA308DBF9901A0F788C7B1912B6
:10168600169AA308DBF91216EC1216CA901A28222B
:10169600E493F622E6438F01538FFDFFC3E583945F
:1016A6001C400122EF857CB7857DB7F0538FFE2263
:1016B600438F02438F01857CB7857DB7901A0DF065
:1016C600538FFC22901A0D7455D19B901A0E74AA52
:1016D600D19B227A3079D07820901A40D196E52095
:1016E600F709A3DAF7227A3079D0901A40E7D19B2E
:1016F60009A3DAF922AB74A875BB01027980BB0293
:10170600027981BB03027982BB04027984BB05029C
:101716007986BB06027992BB07027987BB080279F4
:10172600A3BB0902799CBB0A027988BB0B027989A3
:10173600E8F7227C051205B5DCFB22C2AF1205C50F
:101746001205CC1205D31205DA1205A61205C5122A
:1017560005CC1205D31205DA1205A61205C5120527
:10176600CC1205D31205DAD2AF22C2AF1205DA12B5
:1017760005D31205CC1205C51205A61205DA120507
:10178600D31205CC1205C51205A61205DA1205D329
:101796001205CC1205C5D2AF22AE74AF75C2AF1218
:1017A60005C51205C51205C51205A6DEF21205DA33
:1017B6001205A6DFF8D2AF22F141F139F13975747D
:1017C60001757501757600F19F7C05AD5C1205B556
:1017D600C3ED955C70F5C3E55C9401400AC3E55C16
:1017E60094FF40330217FAD1FBD154F141C2AF75D1
:1017F600EF16F139DCD50576C3E576940350028001
:10180600C61217390575E5741490009F93F808C33E
:10181600E57598500280AD1217391217390574C351
:10182600E574940C50028099120F32121654C2AF0E
:0618360075EF16121739D0
:0319FD0002109441
:101A00000E0915090904FF03FF0903010155AA0185
:101A1000FFFFFFFFFF03FFFFFF25D0285004FF0259
:091A2000007AFF0101000300FF40
:101A4000235467794B463430412320202020202026
:101A500023424C48454C4923463331302320202033
:101A60002020202020202020202020202020202076
:101C0000C2AFC2D353D9BF7581C043B20343FF8073
:101C1000752438752503B1DC7529A5752AF175E29F
:101C20004043F12053A4DF75D4FFD2857DFA7803B9
:101C300079E67C10752200752300901DE97B0675FE
:101C400024987525013085028145208508D8FBD967
:101C5000F9DCF781B7308508D8FBD9F9DCF781B713
:101C6000B19CE493A3C39A6004DDC381B7DBDBB10D
:101C70008E6002812E7B08E493FAA3B16FDBF87AC1
:101C800030B16F752200752300B18EEAFCEBFDC305
:101C9000ED94FE400EB18E8A278B28ED30E0048A49
:101CA000828B83B18E7AC270D8C3ED94FE601950D6
:101CB000CEBD002BEC600F7520007521FF7529004B
:101CC000752A000200008100A827A9280809D80465
:101CD000D90281DCB192EA89AAF281CE0D81A3C337
:101CE000ED94035053EDA2E092007AC5C3E58294CF
:101CF00000E583941C508A200010438F02438F011B
:101D00008529B7852AB7F0300029A827A92808090E
:101D1000438F01538FFDD804D902A133C3E58394C7
:101D20001C4003A3A11689AAE28529B7852AB7F02A
:101D3000A3A116538FFC817F7AC1BD030CE493A34A
:101D4000FAB153DCF8B14B817F8181AA22AB23B178
:101D50006FEBFAEA6222752608C3E52313F523E543
:101D60002213F52250066323A0632201D526EAB18F
:101D7000DCB1DC75260AEAF4200102D285300102CA
:101D8000C285B1DCC3134002C201D526EB22B19259
:101D9000EAFB208502A192308502A197752608AE44
:101DA00024AF25C3EF13FFEE13FEB1E0B1DCC3EAAD
:101DB000133085024480FA30E703632201C3E52330
:101DC00013F523E52213F52250066323A0632201B5
:101DD000D526D9E52265236523F52222AE24AF2539
:101DE0000E0FDEFEDFFCD20122424C48656C6934E6
:071DF000373164F310060116
:00000001FF
